:100000009401242800308A000A30140703188A0A51
:10001000940A82002E3422340034233404342434ED
:100020000834253402342634063427340034283486
:100030000434293408342A3455346E344C346F3443
:1000400063346B34940102280830831685008312D0
:1000500003308316860083124328640089008316C8
:100060000814831208080800880083160815553004
:100070008900AA3089008814640088183C28081177
:10008000831203130800051505164A2102221022C7
:1000900018226C2176210A302D2099000B302D205A
:1000A0009C000C302D209D000D302D209E000E3028
:1000B0002D209F000F302D209A0010302D209B0006
:1000C0008030A00019088D0001300D06031D69283D
:1000D000DC2119088D0001300D06031D7028EF2169
:1000E00019088D0001300D06031D772825221908F7
:1000F0008D0001300D06031D7E28872164308D00A0
:100100008C01640000008C0B81288D0B8128353018
:100110009C0037309D0038309E0020309F0080309A
:10012000A00006189128061C9328003094000512A0
:1001300001309700DC21EF2117088D0001300D06FA
:10014000031DA328392217088D0016300D06031D44
:10015000AA28392217088D0030300D06031DB1285A
:10016000392217088D004A300D06031DB8283922A0
:1001700017088D0063300D06031DBF2839221708AC
:100180008D007D300D06031DC628392217088D000D
:1001900096300D06031DCD28392217088D00B0308A
:1001A0000D06031DD428392217088D00CA300D060C
:1001B000031DDB2839223E2218088D0003300D066E
:1001C0000319E428CE30970018088D0001300D0681
:1001D000031DEB286D2218088D0001300D06031D4C
:1001E000F22825221C08013E9C001C080F399900AA
:1001F00019088D000A300D06031D002930309C00BF
:1002000019088D000A300D06031D09291D08013E3D
:100210009D001D080F39990019088D000A300D0640
:10022000031D142930309D0019088D000A300D0679
:10023000031D1D291E08013E9E001E080F3999004E
:1002400019088D000A300D06031D282930309E0044
:1002500019088D000A300D06031D302931309F002A
:100260001B080A3E9B00CE30170203183929970A53
:100270009A2818088D0001300D06031D402987219A
:10028000051618088D0002300D06031D482949285F
:1002900087284929BA220330831686008312061163
:1002A00086113030B422BA22BA223030B422303033
:1002B000B4222030B4222030B4228030B422030192
:1002C000B4228030B4220301B4221030B4220301DE
:1002D000B422C030B42208000330B4221330B42258
:1002E000BA22BA22BA22BA22BA2208004630A12281
:1002F0007230A1226530A1227130A1222030A122CA
:100300003D30A1222030A1223F30A1220800C03080
:10031000A000013096002030A100DC2101309700C0
:10032000D9210630170203189729970A90295B22D2
:10033000DC2112309400013097000220A100D92165
:10034000063017020318A629970A9D295B22050883
:100350000839990019088D0000300D06031DB229D7
:1003600014309600143016020318B829960A8B2907
:1003700019088D0000300D06031DBF29C2218030F1
:10038000A000080014309400DC21013097002030D8
:10039000A10017088D0005300D020318D129022095
:1003A000A100D921063017020318D829970AC729B6
:1003B00008002108A12208002008B4220301B42269
:1003C000BA22BA22BA22BA22BA2206308D001030DE
:1003D000B4224030B4228D0BE729BA2208001F084E
:1003E000A1221E08A1221D08A1222E30A1221C0834
:1003F000A1222030A1224D30A1224830A1227A3002
:10040000A1220800051504308C0050308D008A228E
:10041000051105308C0010308D008A223222080030
:10042000051108308C0023308D008A22322208000A
:10043000051107308C0008308D008A2208308C00AE
:10044000B0308D008A2232220800051108308C005D
:100450001A088D008A2208308C001B088D008A2221
:1004600032220800051007308C008C0B352A051548
:10047000080002209B0002209A000800013095002D
:1004800050308D008C01640000008C0B432A8D0BD2
:10049000432A06080339980018088D0003300D061A
:1004A0000319542A083095000830150203185A2AF7
:1004B000950A402A080001309500C8308D008C0153
:1004C000640000008C0B602A8D0B602A023015023C
:1004D00003186C2A950A5D2A08000A308900013049
:1004E00034200B3089001C0834200C3089001D0892
:1004F00034200D3089001E0834200E3089001F087A
:1005000034200F3089001A083420103089001B086D
:10051000342008008D0D8F228C0B8A2A0034031C96
:10052000932A0514972A051000000000000000001F
:100530000000000085146400000000000000851029
:1005400000348F00F03908388600061500000611C7
:100550008F0D8F0D8F0D0F0DF039083886000615A1
:1005600000000611BA22003486000615BA220611D0
:10057000BA2200348C0164000000000000008C0BE3
:0A058000BB2A003464006300C22AA5
:02400E00F13F80
:00000001FF
